:1000000016C02DC02CC02BC02AC029C00DC127C0CE
:1000100026C025C024C00000000000FF00FF000033
:10002000FFFFFF0000FF00FFFFFF00FFFFFF1124A5
:100030001FBE20E0A89521BD20E025BFEEECF7E033
:10004000A0E6B0E003C0C89531960D92A036D9F76E
:10005000A0E6B0E001C01D92A837E9F7F0C200C0E9
:100060001895EF92FF920F931F93F92FE82F972F78
:10007000862F042F152FE22EF32EF8940024969548
:1000800087950794969587950794982F802D2FEF45
:1000900030E0732F622F72D3972F862F8083918346
:1000A000912F802F00249695879507949695879594
:1000B0000794982F802D732F622F60D3972F862F50
:1000C000828393839F2D8E2D002496958795079488
:1000D000969587950794982F802D732F622F4ED376
:1000E000972F862F8483958378941F910F91FF908B
:1000F000EF90089580916800282F33278091620047
:10010000909163002817390714F4C19801C0C19A6F
:1001100080916800282F33278091640090916500BA
:100120002817390714F4969801C0969A80916800B0
:10013000282F332780916600909167002817390790
:1001400014F4C09801C0C09A809168008F3310F4F5
:100150008F5F01C080E08093680080916F00282F3E
:1001600033278091690090916A002817390714F4A9
:10017000C49801C0C49A80916F00282F33278091C2
:100180006B0090916C002817390714F4C29801C0D5
:10019000C29A80916F00282F332780916D00909133
:1001A0006E002817390714F4C39801C0C39A8091D0
:1001B0006F008F3310F48F5F01C080E080936F0079
:1001C00080917600282F33278091700090917100E4
:1001D0002817390714F4C79801C0C79A8091760090
:1001E000282F3327809172009091730028173907C8
:1001F00014F4C59801C0C59A80917600282F332742
:1002000080917400909175002817390714F4C698EE
:1002100001C0C69A809176008F3310F48F5F01C0C1
:1002200080E08093760008951F920F920FB60F9290
:1002300011242F933F934F935F936F937F938F93EB
:100240009F93AF93BF93EF93FF9383E882BF809117
:100250007700882351F0C19A969AC09AC49AC29A9C
:10026000C39AC79AC59AC69A01C044DF81E090E05C
:100270009093610080936000FF91EF91BF91AF91E7
:100280009F918F917F916F915F914F913F912F91AE
:100290000F900FBE0F901F90189583E882BF82E0E9
:1002A00083BF89B7826089BF0895482F592F1416DC
:1002B0001506C4F420E030E001C08895809160000C
:1002C00090916100892BC9F3109261001092600037
:1002D0002F5F3F4F2A3031058CF3415050401416A8
:1002E000150644F308958CB381FDFDCF80E190E0C5
:1002F00020D299270895682F792F8CB381FDFDCFE7
:1003000080E190E01ED208958F929F92BF92CF928B
:10031000DF92EF92FF920F931F93CF93DF93882E7C
:10032000992EEE24FF2404E610E0C8ECD0E00F2E56
:10033000F5E0BF2EF02D0F2EF3E0CF2EF02DDD24B3
:100340006894D1F88B2D992787FD9095E80EF91EBA
:100350008C2D992787FD9095080F191F8D2D9927B2
:1003600087FD9095C80FD91FFF201CF4EE24FF24B1
:100370000AC08FEFE816F10439F034F00F2EFFEFCA
:10038000EF2EFF24F02DB194023311051CF402E38B
:1003900010E006C00F3F110521F01CF00FEF10E038
:1003A000C194DD231CF4C0E0D0E006C0CF3FD105EE
:1003B00021F01CF0CFEFD0E0D1942C2F3D2F512F06
:1003C000402F7F2D6E2D82E690E04BDE2C2F3D2FAF
:1003D000512F402F7F2D6E2D89E690E042DE2C2F8D
:1003E0003D2F512F402F7F2D6E2D80E790E039DE7D
:1003F0008114910421F48EE190E057DFA3CF109295
:10040000770080E590E051DF81E08093770080E520
:1004100090E04BDF97CFDF91CF911F910F91FF902D
:10042000EF90DF90CF90BF909F908F9008954F9264
:100430005F926F927F928F929F92AF92BF92CF9274
:10044000DF92EF92FF920F931F93CF93DF93482E8B
:10045000592EF72FE62FB52DA42D8D919C916FEF7E
:1004600070E07AD1882E992E97FCCF96882E992EFF
:10047000082C892C000C881C9908000C881C991CDD
:10048000D52DC42D8A819B816FEF70E065D1C82E78
:10049000D92ED7FCCF96C82ED92E0C2CCD2C000CE3
:1004A000CC1CDD08000CCC1CDD1CD52DC42D8C8192
:1004B0009D816FEF70E050D1D92FC82FD7FDCF9617
:1004C000D92FC82F0C2ECD2F000CCC1FDD0B000C0C
:1004D000CC1FDD1F2E2F3F2F220F331F2E0F3F1F4C
:1004E000F32FE22FEA5EFF4FC895802D682E772408
:1004F000681879080FEF10E0972D862D712F602F67
:100500003DD1662E772EF32FE22FE95EFF4FC8957F
:10051000802DA82EBB24AC18BD089B2D8A2D712FD1
:10052000602F2CD1A62EB72EF32FE22FE85EFF4FBF
:10053000C895802DE82EFF24EC1AFD0A9F2D8E2DE4
:10054000712F602F1BD1E62EF72E01E010E081E025
:1005500090E0ABDE860C971CCA0CDB1CCE0DDF1DB9
:100560002C2F3D2F5D2D4C2D792D682D952D842D13
:1005700078DD0F5F1F4F0F3F110549F344F3DF9103
:10058000CF911F910F91FF90EF90DF90CF90BF9090
:10059000AF909F908F907F906F905F904F90089555
:1005A000CF93DF93C1E0D0E06C2F7D2F82E690E007
:1005B0003EDF6C2F7D2F89E690E039DF6C2F7D2F99
:1005C00080E790E034DF67E070E082E690E02FDFC4
:1005D00067E070E089E690E02ADF67E070E080E79E
:1005E00090E025DF88EE93E060DE6C2F7D2F80E7C2
:1005F00090E01DDF6C2F7D2F89E690E018DF6C2FD7
:100600007D2F82E690E013DF67E070E080E790E006
:100610000EDF67E070E089E690E009DF67E070E0F8
:1006200082E690E004DF88EE93E03FDE2196C7305B
:10063000D1050CF4B9CFB6CFDF91CF910895CFEDAE
:10064000D0E0DEBFCDBF8FEF88BB82BBC19A969A48
:10065000C09AC49AC29AC39AC79AC59AC69A87BBC7
:100660008FE781BB109261001092600010927700BA
:100670002FEF30E0532F422F752F642F82E690E04A
:10068000F0DC2FEF30E0532F422F752F642F89E6D7
:1006900090E0E7DC2FEF30E0532F422F752F642FCF
:1006A00080E790E0DEDCF9DD78948FEE05B6082275
:1006B00005BE80E205B6082A05BE15DE813091052B
:1006C00099F0823091051CF4892B39F028C08230D2
:1006D000910589F00397A1F022C081E090E00BDE44
:1006E00080E090E011DE22C082E090E004DE81E054
:1006F00090E00ADE1BC083E090E0FDDD51DF16C014
:100700008FEF90E0F8DDC1E01092770080E590E097
:10071000CCDDC093770080E590E0C7DDF5CF80E0C9
:1007200090E0E9DD8EE190E0C0DDFCCF80E090E07C
:10073000FFCFE199FECF9FBB8EBBE09A99278DB387
:100740000895E199FECF9FBB8EBB6DBB0FB6F894A9
:10075000E29AE19A0FBE08955527002480FF02C057
:10076000060E571F660F771F6115710521F09695CC
:100770008795009799F7952F802D089597FB092E5F
:1007800007260AD077FD04D00CD006D000201AF43A
:10079000709561957F4F0895F6F7909581959F4FDD
:1007A0000895AA1BBB1B51E107C0AA1FBB1FA617B8
:1007B000B70710F0A61BB70B881F991F5A95A9F70A
:0E07C00080959095682F792F8A2F9B2F089592
:00000001FF
